:0A0EB7000001020203030404050514
:10031900E4F513F512F511F510C203C200C202C2C9
:1003290001120C447E087F008E238F24752B0875DB
:100339002C1275210875221C752908752A4A752DF4
:1003490008752E7890E680E030E70E852125852214
:1003590026852927852A28800C852925852A268509
:100369002127852228EE54E0700302048A751400BF
:100379007515807E087F008E168F17C374FA9FFF4C
:1003890074089ECF2402CF3400FEE48F0F8E0EF541
:100399000DF50CF50BF50AF509F508AF0FAE0EAD25
:1003A9000DAC0CAB0BAA0AA909A808C3120DF6508B
:1003B9002AE515250BF582E514350AF58374CDF088
:1003C900E4FAF9F8E50B2401F50BEA350AF50AE92F
:1003D9003509F509E83508F50880C0E4F50BF50A93
:1003E900F509F508AF0FAE0EAD0DAC0CAB0BAA0AB3
:1003F900A909A808C3120DF65035AE0AAF0BE517C7
:100409002FF582E5163EF583E0FDE5152FF582E52A
:10041900143EF583EDF0E4FAF9F8EF2401F50BEA5F
:100429003EF50AE93509F509E83508F50880B58585
:10043900142385152474002480FF740834FFFEC337
:10044900E52C9FF52CE52B9EF52BC3E5269FF5267C
:10045900E5259EF525C3E5289FF528E5279EF5277F
:10046900C3E5229FF522E5219EF521C3E52A9FF5E3
:100479002AE5299EF529C3E52E9FF52EE52D9EF542
:100489002DD2E843D82090E668E04409F090E65C74
:10049900E0443DF0D2AF90E680E020E105D20712BA
:1004A90007CD90E680E054F7F0538EF8C20330018F
:1004B90005120080C201300329120ECE5024C20356
:1004C900120E0720001690E682E030E704E020E1F2
:1004D900EF90E682E030E604E020E0E4120AD4126C
:0704E9000ED012068A80C745
:0104F00022E9
:1000800090E6B9E0700302015B14700302020424DD
:10009000FE700302029924FB7003020155147003E1
:1000A00002014F147003020143147003020149243A
:1000B000056003020305120ED2400302031190E60D
:1000C000BBE024FE602C14604724FD6016146031F0
:1000D00024067065E52390E6B3F0E52490E6B4F0DD
:1000E000020311E52B90E6B3F0E52C90E6B4F002A4
:1000F0000311E52590E6B3F0E52690E6B4F002039F
:1001000011E52790E6B3F0E52890E6B4F00203117C
:1001100090E6BAE0FF120DB4AA06A9077B01EA49EE
:10012000600DEE90E6B3F0EF90E6B4F002031190AC
:10013000E6A0E04401F002031190E6A0E04401F0E3
:10014000020311120E9A020311120EC102031112C0
:100150000D04020311120E88020311120ED4400383
:1001600002031190E6B8E0247F602B14603C240267
:1001700060030201FAA200E433FF25E0FFA202E4DB
:10018000334F90E740F0E4A3F090E68AF090E68BDE
:100190007402F0020311E490E740F0A3F090E68AC5
:1001A000F090E68B7402F002031190E6BCE0547EFE
:1001B000FF7E00E0D3948040067C007D0180047CBB
:1001C000007D00EC4EFEED4F24B7F582740E3EF537
:1001D00083E493FF3395E0FEEF24A1FFEE34E68F36
:1001E00082F583E0540190E740F0E4A3F090E68AC2
:1001F000F090E68B7402F002031190E6A0E0440157
:10020000F0020311120ED6400302031190E6B8E08B
:1002100024FE601D2402600302031190E6BAE0B4DC
:100220000105C20002031190E6A0E04401F00203C0
:100230001190E6BAE0705990E6BCE0547EFF7E0073
:10024000E0D3948040067C007D0180047C007D002A
:10025000EC4EFEED4F24B7F582740E3EF583E49329
:10026000FF3395E0FEEF24A1FFEE34E68F82F583A5
:10027000E054FEF090E6BCE05480FF131313541FCB
:10028000FFE0540F2F90E683F0E04420F0020311CA
:1002900090E6A0E04401F08078120ED8507390E60A
:1002A000B8E024FE60202402706790E6BAE0B40152
:1002B00004D200805C90E6BAE06402605490E6A04C
:1002C000E04401F0804B90E6BCE0547EFF7E00E00D
:1002D000D3948040067C007D0180047C007D00EC8E
:1002E0004EFEED4F24B7F582740E3EF583E493FF86
:1002F0003395E0FEEF24A1FFEE34E68F82F583E034
:100300004401F0800C1204F1500790E6A0E0440193
:08031000F090E6A0E04480F04B
:0103180022C2
:030033000207FCC5
:0407FC0053D8EF32AD
:100800001201000200000040470502100000010232
:1008100000010A06000200000040010009022E004B
:1008200001010080320904000004FF0000000705F8
:100830000102000200070581020002000705020212
:100840000002000705860200020009022E000101D5
:100850000080320904000004FF00000007050102C7
:100860004000000705810240000007050202400029
:10087000000705860240000004030904100343003A
:100880007900700072006500730073006E0345000C
:100890005A002D0055005300420020004600580029
:1008A000320020004700500049004600200074003C
:1008B0006F00200054004900200035003400310052
:1008C00036002000480050004900200075007300E9
:1008D00069006E00670020004600490046004F0096
:1008E00020005400720061006E007300610063001C
:0C08F000740069006F006E0073000000CF
:1008FC004210B000004110AF00C104C1064210AB61
:10090C000000C105021B00004110AD004110AE00FB
:0B0EAC00E5BB30E7FB90E6F1EFF02221
:100C440090E600E054E74410F000000090E61074D1
:100C5400A0F090E611F000000090E612F000000011
:100C6400E490E613F000000090E61474E0F0000055
:100C740000E490E615F000000090E6047480F000B3
:100C840000007402F00000007406F0000000E4F0BC
:100C940000000090E618F00000007410F00000005E
:100CA40090E61A7408F0000000E490E68DF0120952
:0F0CB400D390E6707401F043B20CD2A8D288221C
:10068A00E5BB30E73FE5AB20E13A75800490E6F43C
:10069A00E070047F0180027F00EF20E0F00000009C
:1006AA0090E6ABE090E6D0F000000090E6ACE09077
:1006BA00E6D1F0000000E4F5BB000000E5BB30E73E
:1006CA00FB0000003004739010ABE07002A3E060FE
:1006DA0069E5BB30E764E5AC20E05F75800490E62D
:1006EA00F4E070047F0180027F00EF20E0F0000058
:1006FA00009010ABE090E6D0F00000009010ACE063
:10070A0090E6D1F000000075BB06000000E5BB30A2
:10071A00E7FB00000090E6AFE0FE90E6B0E07C0068
:10072A002400F51CEC3EF51BC39402500690E648E3
:10073A007406F0E49010ABF0A3F0300609C206D2BA
:10074A00A87F02120A8F9010B0E475F001120DE032
:10075A00AFF0FEBE2727BF10249010AFE0600C7FD9
:10076A0001120788E49010AFF0800B7F01120A8F04
:0E077A009010AF7401F0E49010B0F0A3F022E4
:020ECE00D3222D
:020ED000D3222B
:020ED200D32229
:100D040090E680E030E71800000090E6247402F0DA
:100D1400000000E490E625F0000000D205801600F3
:100D24000000E490E624F000000090E6257440F012
:0D0D3400000000C20590E6BAE0F51DD322D4
:100E880090E740E51DF0E490E68AF090E68B04F0E8
:020E9800D32263
:080EC10090E6BAE0F51AD32215
:100E9A0090E740E51AF0E490E68AF090E68B04F0D9
:020EAA00D32251
:020ED400D32227
:020ED600D32225
:020ED800D32223
:1004F10090E6B9E0244EB409004003020686900557
:1005010006F828287302052102054002055C020550
:100511007802059A0205D602061102063E02065C21
:100521007F0212078890E74074B2F0E490E68AF007
:1005310090E68B04F090E6A0E04480F0020688D2B9
:100541000490E74074B3F0E490E68AF090E68B04FF
:10055100F090E6A0E04480F0020688C20490E740F3
:1005610074B4F0E490E68AF090E68B04F090E6A093
:10057100E04480F0020688E490E68BF0E5BA20E0E2
:10058100FB90E740E0FEA3E07C0024009010ACF07B
:10059100EC3E9010ABF0020688E490E68BF0E5BAF1
:1005A10020E0FB90E6F4E070047F0180027F00EF21
:1005B10020E0F0E4F58090E6C0741EF090E740E0A2
:1005C100FF120EAC90E6C0744EF090E741E0FF12CE
:1005D1000EAC020688E490E68BF0E5BA20E0FB90D1
:1005E100E6F4E070047F0180027F00EF20E0F07507
:1005F100800890E6C0741EF090E740E0FF120EAC58
:1006010090E6C0744EF090E741E0FF120EAC8077A7
:1006110090E6047480F00000007406F0000000E42D
:10062100F000000090E74074B8F0E490E68AF090A2
:10063100E68B04F090E6A0E04480F0804A90E74029
:1006410074B9F0A3E5BBF0E490E68AF090E68B7410
:1006510002F090E6A0E04480F0802C90E74074BA6C
:10066100F090E6D0E090E741F090E6D1E090E742EB
:10067100F0E490E68AF090E68B7403F090E6A0E057
:090681004480F08002D322C32260
:100E2C00C0E0C083C082D2015391EF90E65D7401A3
:080E3C00F0D082D083D0E03237
:100E5C00C0E0C083C0825391EF90E65D7404F0D083
:060E6C0082D083D0E032C9
:100E7200C0E0C083C0825391EF90E65D7402F0D06F
:060E820082D083D0E032B3
:100D7E00C0E0C083C082852925852A2685268285E6
:100D8E002583A37402F08521278522288528828554
:100D9E002783A37407F05391EF90E65D7410F0D0A3
:060DAE0082D083D0E03288
:100E4400C0E0C083C082D2035391EF90E65D740882
:080E5400F0D082D083D0E0321F
:100D4100C0E0C083C08290E680E030E720852125A5
:100D5100852226852682852583A37402F08529278D
:100D6100852A28852882852783A37407F05391EF6C
:0D0D710090E65D7420F0D082D083D0E03297
:010EDA0032E5
:010EDB0032E4
:010EDC0032E3
:010EDD0032E2
:010EDE0032E1
:010EDF0032E0
:010EE00032DF
:010EE10032DE
:010EE20032DD
:010EE30032DC
:010EE40032DB
:010EE50032DA
:010EE60032D9
:010EE70032D8
:010EE80032D7
:010EE90032D6
:010EEA0032D5
:010EEB0032D4
:010EEC0032D3
:010EED0032D2
:010EEE0032D1
:010EEF0032D0
:010EF00032CF
:010EF10032CE
:010EF20032CD
:010EF30032CC
:010EF40032CB
:010EF50032CA
:010EF60032C9
:010EF70032C8
:010EF80032C7
:010EF90032C6
:010EFA0032C5
:010EFB0032C4
:010EFC0032C3
:010EFD0032C2
:10078800EF30E00D908100E09010ADF0A3E054FE52
:10079800F0EF30E10D909100E09010ADF0A3E0543F
:1007A800FDF0EF30E20D90A100E09010ADF0A3E075
:1007B80054FBF0EF30E30D90B100E09010ADF0A3E2
:0507C800E054F7F022EF
:100A8F00EF30E00D908000E09010ADF0A3E0440156
:100A9F00F0EF30E10D909000E09010ADF0A3E04446
:100AAF0002F0EF30E20D90A000E09010ADF0A3E067
:100ABF004404F0EF30E30D90B000E09010ADF0A3E0
:050ACF00E04408F022E4
:03000300020EC921
:050EC900D206C2A832B0
:03004300020B00AD
:03005300020B009D
:100B0000020E2C00020E7200020E5C00020E440067
:100B1000020D7E00020D4100020EDA00020EDB0023
:100B2000020EDC00020EDD00020EDE00020EDF000F
:100B3000020EE000020EE100020EE200020EE300EF
:100B4000020EE400020EDB00020EE500020EE600DB
:100B5000020EE700020EE800020EE900020EEA00B3
:100B6000020EEB00020EDB00020EDB00020EDB00C9
:100B7000020EEC00020EED00020EEE00020EEF007F
:100B8000020EF000020EF100020EF200020EF3005F
:100B9000020EF400020EF500020EF600020EF7003F
:100BA000020EF800020EF900020EFA00020EFB001F
:080BB000020EFC00020EFD0024
:100AD40090E682E030E004E020E60B90E682E0302D
:100AE400E119E030E71590E680E04401F07F147EE0
:0C0AF40000120CC390E680E054FEF022DB
:100E070090E682E044C0F090E681F043870100005D
:040E170000000022B5
:1007CD0030070990E680E0440AF0800790E680E06B
:1007DD004408F07FDC7E05120CC390E65D74FFF0DB
:0F07ED0090E65FF05391EF90E680E054F7F02232
:020DB400A9078D
:100DB600AE2DAF2E8F828E83A3E064037017AD0134
:100DC60019ED7001228F828E83E07C002FFDEC3EB0
:090DD600FEAF0580DF7E007F0006
:010DDF0022F1
:100CC3008E188F1990E600E05418700DE518C313C1
:100CD300F518E51913F519801590E600E05418FF8F
:100CE300BF100BE51925E0F519E51833F518E519DB
:100CF3001519AE18700215184E6005120E1B80EE02
:010D030022CD
:100E1B007400F58690FDA57C05A3E582458370F9EA
:010E2B0022A4
:10091C006080100001013F0101010107000201008C
:10092C0000000000020002020202020700000000A8
:10093C000000003F01013F0101010107000201001D
:10094C00000000000604060606060607000000006C
:10095C000000003F01010101013801070000020005
:10096C00020100000301070507070707000000004C
:10097C00002D003F010101010138010700020402B2
:10098C00040100000200060406070707000000002F
:10099C00002D003F602410870000000000000000C4
:1009AC00000000000000000000000000000000003B
:1009BC00000000000000000000000000471080E074
:0609CC00000007CE4E0002
:1009D30090E60174CEF090E6F574FFF0901080E09D
:1009E30090E6F3F0901081E090E6C3F0901082E07F
:1009F30090E6C1F0901083E090E6C2F0901085E09D
:100A030090E6C0F0901086E090E6F4F075AF0774BE
:100A130010F59A7400F59B759DE4E4F59EFF90E64E
:100A23007BE090E67CF00FBF80F490E67174FFF0FA
:100A3300F5B490E672E04480F043B680000000E431
:100A430090E6C4F000000090E6C5F0901087E090B7
:100A5300E6C6F0901088E090E6C7F0901089E09029
:100A6300E6C8F090108AE090E6C9F090108BE09011
:100A7300E6CAF090108CE090E6CBF090108DE090F9
:0B0A8300E6CCF090108EE090E6CDF085
:010A8E002245
:03000000020BB838
:0C0BB800787FE4F6D8FD75812E020BFF5B
:100DE000C5F0F8A3E028F0C5F0F8E582158270029E
:060DF0001583E038F0223B
:100DF600EB9FF5F0EA9E42F0E99D42F0E89C45F053
:010E060022C9
:100BC400020319E493A3F8E493A34003F68001F22B
:100BD40008DFF48029E493A3F85407240CC8C33332
:100BE400C4540F4420C8834004F456800146F6DF01
:100BF400E4800B01020408102040809008FCE47E8D
:100C0400019360BCA3FF543F30E509541FFEE493F5
:100C1400A360010ECF54C025E060A840B8E493A3BC
:100C2400FAE493A3F8E493A3C8C582C8CAC583CAE7
:100C3400F0A3C8C582C8CAC583CADFE9DEE780BE9F
:0109D2000024
:00000001FF
